:100000000C94D3040C941B050C941B050C941B0539
:100010000C941B050C941B050C941B050C941B05E0
:100020000C941B050C941B050C949D1D0C941B0536
:100030000C94741D0C941B050C941B050C941B054F
:100040000C941B050C941B050C941B050C941B05B0
:100050000C941B050C944E1D0C941B050C941B0555
:100060000C941B050C941B050C941B050C941B0590
:100070000C941B050C941B050C941B050C941B0580
:100080000C941B050C941B050C941B050C941B0570
:100090000C941B050C941B050C941B050C941B0560
:1000A0000C941B050C941B050C941B050631FF09D1
:1000B00074A1010975150026FF00952075088102BD
:1000C0000976150026FF00952075089102C00501EC
:1000D0000902A1010901A1008501050919012908E9
:1000E00015002501950875018102050109300931C6
:1000F0001581257F95027508810609381581257FB0
:10010000950175088106050C0A38021581257F9531
:100110000175088106C0C005010980A1018502168C
:1001200001002637001A81002AB700751095018159
:1001300000C0050C0901A1018503160100269C02DF
:100140001A01002A9C02751095018100C005010961
:1001500006A101050719E029E71500250195087595
:10016000018102950175088101050819012905958C
:100170000575019102950175039101050719002983
:10018000FF150026FF00950675088100C02831295B
:100190000A002832290A002833290A002834290AAB
:1001A000005D0A0025303258005B006D6F64656C9D
:1001B0003A20253032580A000A0025303258006DA6
:1001C000303131305F73656E64206572723A2000A1
:1001D0000A0025303258006D303131305F7265636E
:1001E00076206572723A20002000253032580025B2
:1001F000583A2530386225730A000A2020303132FF
:1002000033343536370A004C45443A2025303258CD
:100210000A000A4C6F6F702073746172742E0A00AA
:100220000A55534220636F6E666967757265642E66
:100230000A000A544D4B3A3264643934382F4C5515
:1002400046413A6436613764660A00090254000385
:100250000100A0320904000001030101000921117D
:100260000100012240000705810308000A0904017A
:10027000000103010200092111010001227F000792
:1002800005820308000109040200010300000009BF
:100290002111010001222200070583032000011221
:1002A00001100100000008EDFE1001010101020033
:1002B0000132034D00300031003100300020006B6E
:1002C000006500790062006F006100720064002028
:1002D0000063006F006E00760065007200740065B8
:1002E00000720000000E0374002E006D002E006BE3
:1002F000002E0000000403090473797374656D3ADD
:1003000020253034580A00636F6E73756D65723A3C
:1003100020253034580A003F004D3E2000433E2047
:10032000000A00257500363A20776865656C5F74B1
:10033000696D655F746F5F6D61783A20000A002512
:100340007500353A20776865656C5F6D61785F731D
:10035000706565643A20000A00257500343A2074FF
:10036000696D655F746F5F6D61783A20000A0025E2
:100370007500333A206D61785F73706565643A206B
:10038000000A00257500323A20696E746572766144
:100390006C286D73293A20000A00257500313A2037
:1003A00064656C6179282A31306D73293A20000A1E
:1003B000092D2056616C756573202D0A004D3E0095
:1003C0004D25643E20003F007365742064656661BE
:1003D000756C740A00433E20000A00253032582014
:1003E000006B6579626F6172643A20000416070938
:1003F0000B0A1D1B06196405141A08151C171E1F6D
:10040000202123222E26242D25273012182F0C13CD
:10041000280F0D340E333136381110372B2C352A76
:100420007F80807B79397A808080808080634F8074
:10043000808050535180808058525780808062590C
:100440005A5B5C5D5E5F80606180808080805680EA
:10045000808066805480808080558080290A0025B5
:1004600075002F002575005D2800256400200025FB
:100470006400200025640020002564007C002530F5
:100480003258006D6F7573656B6579205B62746EB1
:100490007C782079207620685D287265702F6163F2
:1004A0006C293A205B000A092D204D6167696320A1
:1004B0002D0A643A0964656275670A783A096465C9
:1004C000627567206D61747269780A6B3A096465B8
:1004D000627567206B6579626F6172640A6D3A09B3
:1004E0006465627567206D6F7573650A763A097683
:1004F000657273696F6E0A733A0973746174757308
:100500000A633A09636F6E736F6C65206D6F646583
:100510000A302D343A096C61796572302D342846E1
:1005200031302D4634290A506175733A09626F6F74
:10053000746C6F616465720A000A092D20436F6E46
:10054000736F6C65202D0A4553432F713A097175FD
:1005500069740A6D3A096D6F7573656B65790A0088
:100560003F0074696D65725F72656164333228297A
:100570003A202530346C580A006B6579626F6172DD
:10058000645F69646C653A2025580A006B6579627E
:100590006F6172645F70726F746F636F6C3A202565
:1005A000580A00686F73745F6B6579626F6172647B
:1005B0005F6C65647328293A2025580A000A092DC2
:1005C00020537461747573202D0A004743433A2009
:1005D000372E332E30204156522D4C4942433A207B
:1005E000322E302E30204156525F415243483A203D
:1005F000617672350A004F5054494F4E533A204CA1
:10060000554641204D4F5553454B4559204558546B
:1006100052414B455920434F4E534F4C4520434F79
:100620004D4D414E44204B45594D41505F5345433C
:1006300054494F4E20343039360A004255494C4413
:100640003A20326464393438202831323A30343A2E
:100650003337204A616E2033302032303233290A5A
:10066000005649443A2030784645454428742E6D5A
:100670002E6B2E29205049443A20307830313130C9
:10068000284D30313130206B6579626F61726420A2
:10069000636F6E76657274657229205645523A20F2
:1006A0003078303130310A00444553433A20636F8B
:1006B0006E76657274204D30313130206B65796211
:1006C0006F61726420746F205553420A000A092D2D
:1006D0002056657273696F6E202D0A000A6D6F7562
:1006E00073653A206F66660A000A6D6F7573653A26
:1006F000206F6E0A000A6B6579626F6172643A203E
:100700006F66660A000A6B6579626F6172643A20EF
:100710006F6E0A000A6D61747269783A206F6666BE
:100720000A000A6D61747269783A206F6E0A000AD5
:1007300064656275673A206F6E0A000A64656275C7
:10074000673A206F66660A000A0A626F6F746C6F00
:10075000616465722E2E2E2000433E20006D6B5F7B
:10076000776865656C5F74696D655F746F5F6D61F7
:1007700078203D2025640A006D6B5F776865656CA5
:100780005F6D61785F7370656564203D2025640A44
:10079000006D6B5F74696D655F746F5F6D6178206C
:1007A0003D2025640A006D6B5F6D61785F73706535
:1007B0006564203D2025640A006D6B5F696E746579
:1007C0007276616C203D2025640A006D6B5F646564
:1007D0006C6179203D2025640A006D6B5F77686548
:1007E000656C5F74696D655F746F5F6D6178203DE6
:1007F0002025640A006D6B5F776865656C5F6D61CD
:10080000785F7370656564203D2025640A006D6B18
:100810005F74696D655F746F5F6D6178203D202541
:10082000640A006D6B5F6D61785F7370656564204D
:100830003D2025640A006D6B5F696E746572766198
:100840006C203D2025640A006D6B5F64656C6179E6
:10085000203D2025640A0077686572652064656C18
:1008600074613A20637572736F723D25642C207732
:100870006865656C3D25640A53656520687474700D
:100880003A2F2F656E2E77696B6970656469612EEA
:100890006F72672F77696B692F4D6F7573655F6B2B
:1008A0006579730A000A092D204D6F7573656B65B4
:1008B00079202D0A4553432F713A09717569740ADD
:1008C000313A0964656C6179282A31306D73290ADF
:1008D000323A09696E74657276616C286D73290A03
:1008E000333A096D61785F73706565640A343A095B
:1008F00074696D655F746F5F6D61780A353A097769
:100900006865656C5F6D61785F73706565640A36F4
:100910003A09776865656C5F74696D655F746F5FD0
:100920006D61780A0A703A097072696E7420766196
:100930006C7565730A643A09736574206465666151
:10094000756C74730A75703A092B310A646F776E8F
:100950003A092D310A706775703A092B31300A70E7
:1009600067646F776E3A092D31300A0A73706565D6
:1009700064203D2064656C7461202A206D61785F7D
:100980007370656564202A20287265706561742023
:100990002F2074696D655F746F5F6D6178290A003F
:1009A0004C25640A000011241FBECFEFDAE0DEBF41
:1009B000CDBF04B603FE28C0809146039091470343
:1009C000A0914803B09149038730904BA740B04BAA
:1009D000D9F41092460310924703109248031092E4
:1009E000490314BE0FB6F894A89580916000886101
:1009F00080936000109260000FBE10920108109268
:100A00000008E0E0F8E3099511E0A0E0B1E0EEE0D5
:100A1000F5E402C005900D92A433B107D9F723E0A5
:100A2000A4E3B1E001C01D92A634B207E1F70E9431
:100A3000771E0C9485220C940000FF93EF93E091B5
:100A40003401F0913501309709F00995EF91FF914C
:100A50000895FC018591803011F0EFDFFBCF089500
:100A6000FF27E0E230E247FF0CC0419597FF09C045
:100A7000EDE26095709580959095611D711D811DC9
:100A8000911D27FF02C0219530E350E2AA27660F8F
:100A9000771F881F991FAA1FA41710F0A41B639526
:100AA0005A95A9F7AA3008F0A95FA05DAF93F39516
:100AB000611571058105910541F7ED3211F4EF9350
:100AC000F395F21718F43F93F395FBCF8F91B5DFB1
:100AD000FA95E1F70895E991F9918591803021F037
:100AE000853219F0AADFF9CF089520E0E8945591F6
:100AF0005532C1F3503311F4689455915A3348F488
:100B0000505390F3220F022E220F220F200D250F9B
:100B1000F4CF0EF4219589919991533619F35337F7
:100B200029F1533559F1BC0188279927E8945C369F
:100B300021F48991999168945591543639F446EF8E
:100B40007EF077FF0DC08FEF9FEF0AC055374AE068
:100B500039F0583540E121F0523642E009F008956D
:100B6000FF93EF937DDFEF91FF91B7CFFF93EF936B
:100B7000FC0181918030B9F360DFFBCFFF93EF93ED
:100B800068DFF1CFDF93CF93CDB7DEB72596A3DF34
:100B9000CF91DF9108958091300380FF0CC0609168
:100BA000140170E0759567957595679561157105E8
:100BB00049F1862F089581FF06C06091140170E00D
:100BC00075956795F3CF6091140182FD0BC09091EC
:100BD00031039923A1F060911301809114019617BC
:100BE00038F0682F70E06038710500F38FE70895E2
:100BF000899FC001112470E00E945722F4CF61E068
:100C000070E0D7CF81E008958091300380FF12C05B
:100C10006091160185E0689FB00111247595679574
:100C20007595679560387105A8F561157105A1F195
:100C3000862F089581FF09C06091160185E0689FA5
:100C4000B001112475956795EDCF82FF07C06091C3
:100C5000160185E0689FB0011124E4CF2091310393
:100C60002223A9F0909115016091160185E0689FFB
:100C7000B00111242917B0F6269FA001279F500D1F
:100C80001124692F70E0CA010E945722CBCF65E082
:100C900070E0CECF8FE7089581E0089528E0729F3D
:100CA000F0011124E60FF11DE451FC4F6491E62F91
:100CB000E295E77028E0829FC00111248E0F911DFC
:100CC00024E0880F991F2A95E1F7E62FEF70E80FCF
:100CD000F92FF11DEE0FFF1FE050F8498591949117
:100CE00008952FB7F89480913B0390913C03A09115
:100CF0003D03B0913E032FBF0895E6E3F2E09281F9
:100D0000891301C01282319692E0EC33F907B9F7EA
:100D10000895A8E3B2E0EFEF90E02D91821751F033
:100D2000EF3F19F4211101C0E92F9F5F9630A9F719
:100D3000EF3F09F408950E2E000CFF0BEA5CFD4F07
:100D4000828308954F925F926F927F929F92AF92AB
:100D5000BF92CF92DF92EF92FF920F931F93CF93A8
:100D6000DF9300D000D01F92CDB7DEB76B837C83BA
:100D70008D837A018C819D81892B49F08FEFF81248
:100D800004C081E09FEF491719F080E001C081E0C5
:100D900080FD6AC00F2D10E0CE2CD12C8B818823D2
:100DA00009F456C04090B8025090B9026090BA025F
:100DB0007090BB028091420390914303A091440341
:100DC000B0914503482A592A6A2A7B2A2FE1A22E8C
:100DD000B12C9A2CD301C2010A2C04C0B695A79558
:100DE000979587950A94D2F780FD2BC081E0A81AC9
:100DF000B10878F7912CF80193E0EE0FFF1F9A9558
:100E0000E1F7E454FD4FEC0DFD1D9082E982FA827A
:100E100069817A81892D0F900F900F900F900F901C
:100E2000DF91CF911F910F91FF90EF90DF90CF90C6
:100E3000BF90AF909F907F906F905F904F900C9479
:100E40004E06B7018A2D0E944E06019779F2D3CF44
:100E5000F80183E0EE0FFF1F8A95E1F7E454FD4FA0
:100E6000EC0DFD1D9080D2CF90E080E00F900F90B0
:100E70000F900F900F90DF91CF911F910F91FF90E6
:100E8000EF90DF90CF90BF90AF909F907F906F904A
:100E90005F904F90089541E050E060E070E004C042
:100EA000440F551F661F771F8A95D2F740955095BE
:100EB000609570958091B8029091B902A091BA02A4
:100EC000B091BB0284239523A623B7238093B80255
:100ED0009093B902A093BA02B093BB02089541E087
:100EE00050E060E070E004C0440F551F661F771F9C
:100EF0008A95D2F78091B8029091B902A091BA0276
:100F0000B091BB02842B952BA62BB72B8093B802F4
:100F10009093B902A093BA02B093BB020895809156
:100F2000B70290918602981301C008958F5F877071
:100F3000FACF1F93CF93DF9300D000D01F92CDB78D
:100F4000DEB7942F4983252F5A836B837C838D834F
:100F50004C815D8181E0452B31F02F3F19F481E018
:100F60009F3F09F080E0182F117080FD2CC049814F
:100F70005A816B817C818D810E94A206292F229546
:100F80002F702C3078F42A30A8F422502230C8F088
:100F9000812F0F900F900F900F900F90DF91CF91B6
:100FA0001F9108952C3011F02F3091F793FB1127EA
:100FB00010F9EECF803C28F0803E50F3815F833003
:100FC00038F311E0E5CF10E0E3CFE0913203F09188
:100FD0003303309721F00190F081E02D099480E0F7
:100FE0000895E8EDF0E080818E7F80831092E2002A
:100FF0001092DA001092E100A0EEB0E08C918160D6
:101000008C9380818F77808319BCA7EDB0E08C91A1
:101010008E7F8C9380818F7E8083109264020895EE
:101020000E94F107F89487E797E79093010880936F
:10103000000887E090EBDC01809346039093470320
:10104000A0934803B093490388E19CE00FB6F8945D
:10105000A895809360000FBE90936000FFCFFC01C5
:10106000809178029091790286179707A0F0611518
:10107000710529F49091E8009E779093E80090E044
:101080006115710551F4911108C08091E80082FF4B
:1010900035C080E00895BC01F2CF80917A028823A8
:1010A000C9F18530C9F18091E80083FD31C080919C
:1010B000E80082FDEACF8091E80080FFE1CF209137
:1010C000F3008091F200322F282F6115710519F07D
:1010D0002830310558F091E02830310509F090E0D2
:1010E0002091E8002E772093E800CACF8191809369
:1010F000F100615071092F5F3F4FE7CF80917A0275
:10110000882341F0853041F08091E80083FFBDCF16
:1011100081E0089582E0089583E008952091E4003D
:101120003091E50085E69091EC0090FF06C090912B
:10113000E80090FF06C080E008959091E80092FDDD
:10114000FACF90917A02992391F0953091F0909195
:10115000EB0095FD10C04091E4005091E50024178C
:10116000350709F381509A01F1F684E0089582E091
:10117000089583E0089581E008958091720287FFC9
:1011800013C08091E80082FF06C08091E8008B7751
:101190008093E80004C080917A028111F2CF089513
:1011A00080917A028823D9F38091E80080FFF8CFFC
:1011B0008091E8008E77ECCF982F9093E900242F50
:1011C000762F50E0891731F07091EC002091ED00FE
:1011D0005091F00021FD07C09F5F973071F7809319
:1011E000E90081E008953091EB003E7F3093EB0001
:1011F0003091ED003D7F3093ED003091EB00316098
:101200003093EB007093EC002093ED005093F000CE
:101210002091EE0027FDE0CF80E00895CF92DF928D
:10122000EF92FF920F931F93CF93DF93C8EDD0E01F
:1012300088818F7E8883E7EDF0E080818160808304
:1012400084E082BF81E08093640288818E7F8883FE
:1012500002EE10E0F80110821092DA0081EEC82E42
:10126000D12CF601108288818F77888388818068ED
:10127000888388818F7D888319BC10927A021092AE
:1012800071021092700210926F0290EEE92EF12C12
:10129000F70180818B7F808388818160888342E031
:1012A00060E080E00E94DC08F60180818E7F808310
:1012B000F801808181608083808188608083F7016C
:1012C00080818E7F8083888180618883DF91CF9148
:1012D0001F910F91FF90EF90DF90CF900895809134
:1012E0006602089580914202811113C09FB7F8945D
:1012F00040913B0350913C0360913D0370913E034C
:101300009FBF443C59406105710518F081E080930E
:1013100042020895EF92FF920F931F93CF93DF93B2
:10132000D82F0FB607FE46C080917A02843079F03C
:101330008091040190E001962091060130E0822323
:101340009323209105012817190609F0CDC00E94AA
:10135000720981110FC08091040190E001962091E3
:10136000060130E0822393232091050128171906F6
:1013700009F0BAC00E9471068C01C091E900CF70DB
:101380008091EC0080FD37C080E0C82B83E0809323
:10139000E90085E0E82E8091EB0085FD08C0809192
:1013A000EB0080FF04C08091EE0087FD44C0CF7049
:1013B000C093E900E09104018E2F90E00196209106
:1013C000060130E082239323209105012817190696
:1013D00009F482C08091020190910301E80FF92F76
:1013E000F11DD083809104018F5F909106018923C4
:1013F0008093040171C080E8C8CFE0910201F091B0
:101400000301E80FF11D90818F5F20910601822377
:10141000809305019093F1008091E80085FD0BC059
:101420008091E80080FF07C08091E8008E7780936C
:10143000E800E09201018091050190910401981764
:1014400041F19091E80095FDD8CF80E029C010923D
:10145000F10032C08091040190E0019620910601D4
:1014600030E082239323209105012817190609F003
:101470009ECFF0900101FF2009F499CF0E947106E0
:101480008017910709F487CFFA94F09201018C013B
:1014900082CF8091E80085FFD8CFD093F10081E022
:1014A0002091F3009091F200322F292F232B79F015
:1014B0009091E80090FF0BC09091E80095FDC7CF98
:1014C0009091E8009E779093E800E09201018823D4
:1014D00009F2CF70C093E90080E0DF91CF911F91B6
:1014E0000F91FF90EF900895E091040173CF509811
:1014F000589A08955898509A08955198599A08956D
:101500008B3749F08F3F39F0282F30E035952795FC
:101510002F738078822B08958330C9F128F48130AD
:1015200061F0823019F10895853009F452C008F451
:101530003FC0863009F45EC0089580911801681795
:1015400090F4861B80931801809118011F928F934D
:1015500088E498E09F938F930E94C2050F900F90AC
:101560000F900F90089510921801EECF80911701FF
:10157000681750F4861B80931701809117011F9202
:101580008F9386E398E0E6CF10921701F6CF809113
:101590001601681750F4861B80931601809116017E
:1015A0001F928F9383E298E0D5CF10921601F6CF69
:1015B00080911501681750F4861B80931501809166
:1015C00015011F928F938EE098E0C4CF1092150101
:1015D000F6CF80911401681750F4861B8093140194
:1015E000809114011F928F9385EF97E0B3CF1092F3
:1015F0001401F6CF80911301681750F4861B809375
:101600001301809113011F928F938AED97E0A2CF6F
:1016100010921301F6CF833009F445C028F48130CD
:1016200061F0823049F10895853009F46AC008F408
:1016300051C0863009F47CC0089580911801482F6C
:10164000460F5527551F4F3F510594F4680F60937F
:101650001801809118011F928F938BEC97E09F9354
:101660008F930E94C2050F900F900F900F900895D6
:101670008FEF80931801EDCF80911701482F460F0F
:101680005527551F4F3F510554F4680F60931701BC
:10169000809117011F928F9389EB97E0E0CF8FEF36
:1016A00080931701F5CF80911601482F460F5527DB
:1016B000551F4F3F510554F4680F609316018091F8
:1016C00016011F928F9386EA97E0C9CF8FEF809320
:1016D0001601F5CF80911501482F460F5527551F4C
:1016E0004F3F510554F4680F609315018091150127
:1016F0001F928F9381E997E0B2CF8FEF809315010E
:10170000F5CF80911401482F460F5527551F4F3FA5
:10171000510554F4680F60931401809114011F92D5
:101720008F9388E797E09BCF8FEF80931401F5CFDD
:1017300080911301482F460F5527551F4F3F5105E4
:1017400054F4680F60931301809113011F928F93DB
:101750008DE597E084CF8FEF80931301F5CFCF9382
:10176000DF9320917D0230917E022817390701F125
:1017700090937E0280937D02E0913203F0913303D7
:101780003097B1F0EC010084F185E02D099580914E
:1017900041038570853061F4DF93CF9387E093E058
:1017A0009F938F930E94C2050F900F900F900F9000
:1017B000DF91CF910895CF93DF9320917B023091F9
:1017C0007C022817390701F190937C0280937B02F9
:1017D000E0913203F09133033097B1F0EC010680D1
:1017E000F781E02D0995809141038570853061F482
:1017F000DF93CF9389EF92E09F938F930E94C2056E
:101800000F900F900F900F90DF91CF91089585EA80
:1018100098E00E9429051F9281E08F931F9285E036
:101820008F9387E598E09F938F930E94C2050F9056
:101830000F900F900F900F900F900895CF9380917D
:10184000410383FF7EC083E894E00E9429058091D4
:1018500036031F928F938EE794E09F938F930E949D
:10186000C2058CE794E00E94290580913703282F58
:10187000082E000C330B3F938F9389E794E09F93DE
:101880008F930E94C20587E794E00E94290580910A
:101890003803282F082E000C330B3F938F9384E7D7
:1018A00094E09F938F930E94C20582E794E00E9488
:1018B000290580913903282F082E000C330B3F9304
:1018C0008F938FE694E09F938F930E94C2058DE6DD
:1018D00094E00E94290580913A03282F082E000CDD
:1018E000330B3F938F938AE694E09F938F930E94EC
:1018F000C20587E694E00E942905809131031F927A
:101900008F9384E694E09F938F930E94C20582E6B2
:1019100094E00E942905809130031F928F938FE5F8
:1019200094E09F938F930E94C2058CE594E00E94FF
:1019300029058DB79EB74C960FB6F8949EBF0FBE83
:101940008DBFE0913203F0913303309751F0C09195
:1019500036030480F581E02D86E393E00995C0937A
:1019600036030E9471069093350380933403CF9120
:1019700008950F931F93CF93DF9380912E0390913F
:101980002D03892B8093360290912C03992389F0A3
:10199000892B80933602E7E3F2E02EE332E080E029
:1019A000919191118F5F2E173F07D1F781111092FE
:1019B0002C03E0913203F09133033097B1F10280B0
:1019C000F381E02D86E392E009958091410382FF47
:1019D0002CC080FF04C081EE93E00E942905D0E076
:1019E000C0E00BED13E08091410380FF0EC0FE01CB
:1019F000EA5CFD4F80811F928F931F930F930E948B
:101A0000C2050F900F900F900F902196C830D1050E
:101A100051F78091410380FF08C089ED93E0DF9189
:101A2000CF911F910F910C942905DF91CF911F91B8
:101A30000F91089510922E0310922D03E6E3F2E029
:101A400011821282138214821582168217820E94DA
:101A5000B90C85E0E6E3F3E0DF011D928A95E9F732
:101A600010923103109230030E941E0C90E080E02F
:101A70000E94DB0B90E080E00C94AF0BCF93C82F5B
:101A80001F928F9380EA99E09F938F930E94C205E3
:101A900081E090E0A0E0B0E004C0880F991FAA1F89
:101AA000BB1FCA95D2F78093420390934303A09340
:101AB0004403B09345030F900F900F900F90CF9178
:101AC0000C941A0D0F931F93CF93DF93CDB7DEB70E
:101AD000AA970FB6F894DEBF0FBECDBF80917A02F1
:101AE000882309F452C11091E9001F708091EC0025
:101AF00080FF39C080E8182B1092E9008091E8003F
:101B000083FF40C1E2E7F2E08AE792E02091F10032
:101B100021938E179F07D1F780917302833009F4C8
:101B200070C018F5813009F447C0823009F4DEC076
:101B30008091E80083FF18C1809172029091730236
:101B40009A3008F011C1E92FF0E0E755F24F0C94FC
:101B50006B22870EAD0EB40EAD0EB40E0F0F310F0B
:101B6000B40E30103D1080E0C6CF8A3009F4ADC00D
:101B70008B3009F47DC08930D9F6809172028132B0
:101B8000B9F68091760290917702892B89F680913F
:101B9000E800877F8093E8008091E80082FF2CC0F6
:101BA0008091F100809366028091E8008B778093AA
:101BB000E8000E94BD08BCCF80917202813A09F012
:101BC000B7CF8091E800877F8093E800809176020C
:101BD00090917702892B61F060E090E080E070E006
:101BE0000E942F088091E8008B778093E800A0CFB7
:101BF00068E087E692E0F3CF80917A028111CCCF42
:101C000097CF80917202813A09F092CF809176024B
:101C100090917702892BA1F48091E800877F8093CF
:101C2000E8008091E80080FFFCCF80911201809352
:101C3000F1008091E8008E778093E8000E94BD0853
:101C40008091760290917702019709F071CF80918F
:101C5000E800877F8093E8008091E80080FFFCCF58
:101C6000809111018093F1008091E8008E779FCFE1
:101C700080917202813209F05BCF8091760290915F
:101C80007702892B69F48091E800877F8093E800D0
:101C90000E94BD0880917402809312010E941A0D67
:101CA0008091760290917702019709F041CF80915F
:101CB000E800877F8093E8000E94BD08809174024D
:101CC000809311010E941A0D33CF809172028132EC
:101CD00009F02ECF8091E800877F8093E8000E9472
:101CE000BD088091750280933F0322CF80917202DC
:101CF000813A09F01DCF8091E800877F8093E8004A
:101D00008091E80080FFFCCF80913F03ABCF80380B
:101D100089F0823849F5809176028F70873020F5FE
:101D20008093E9008091EB0085FB882780F9109271
:101D3000E90006C080916F0290917002911182605B
:101D40009091E800977F9093E8008093F1001092C3
:101D5000F1008091E8008E7731C0282F2D7F21F48B
:101D60008823F1F0823079F18091E80083FF0AC086
:101D70008091E800877F8093E8008091EB0080628B
:101D80008093EB001F701093E900AA960FB6F894A9
:101D9000DEBF0FBECDBFDF91CF911F910F91089590
:101DA00080917402813001F7933009F080E08093D4
:101DB00070021092E9008091E800877F8093E8002C
:101DC0000E94BD08D1CF809174028111F2CF809121
:101DD00076028F702FEF280F263030F68093E900BF
:101DE0002091EB0020FFE5CF933031F48091EB00A0
:101DF00080628093EB00DDCF9091EB009061909337
:101E0000EB0021E030E001C0220F8A95EAF7209331
:101E1000EA001092EA008091EB008860EACF81111D
:101E2000A3CF009174020F778091E3008078802B1C
:101E30008093E3008091E800877F8093E8000E9410
:101E4000BD088091E80080FFFCCF8091E3008068AE
:101E50008093E30083E0011101C082E080937A0265
:101E600083CF8058823008F07FCF20917402309168
:101E700075022C3D83E03807A1F583E08A838AE26E
:101E800089834FB7F894DE01139620E03EE051E2DB
:101E9000E32FF0E050935700E49120FF03C0E29558
:101EA000EF703F5FEF708E2F90E0EA30C0F0C79682
:101EB0008D939D932F5F243159F74FBF8091E80098
:101EC000877F8093E8006AE270E0CE0101960E946D
:101ED0002F088091E8008B778093E80045CFC0966B
:101EE000E7CF8091760290917702432F55274330B8
:101EF000510509F44FC078F54130510509F445C04A
:101F000084E590E0EBE4F2E04230510509F02CCF9B
:101F10002091E800277F2093E800209178023091FB
:101F200079028217930708F49C0140E021153105DE
:101F300009F063C0411161C08091E80082FDC9CF02
:101F400080917A02882329F2853019F28091E80085
:101F500083FFF2CFBECF4132510509F43FC0423278
:101F6000510509F001CF8330910508F0FDCEFC0149
:101F7000EE0FFF1FE35EFE4F0190F081E02D865EC5
:101F80009E4FDC018C9190E01DC082E190E0EFE972
:101F9000F2E0BECF332721303105C1F060F02230AE
:101FA000310509F0E1CEE1EBF2E0E4918E2F90E013
:101FB000E1EBF2E007C0E5EFF2E0E4918E2F90E074
:101FC000E5EFF2E0009709F4CFCEA2CFE5EEF2E024
:101FD000E4918E2F90E0E5EEF2E0F4CF83309105AE
:101FE00008F0C2CE880F991FFC01ED5DFE4F0190F5
:101FF000F081E02D89E090E08BCF80917A028823F8
:1020000009F467CF853009F464CF8091E80083FD3F
:1020100060CF8091E80082FD8FCF8091E80080FF43
:1020200085CF8091F3009091F20089279827892726
:102030002115310519F08830910550F041E00897DD
:1020400009F040E08091E8008E778093E8006ECF41
:1020500044914093F1003196215031090196E8CF27
:10206000803809F081CE8091E800877F8093E80076
:10207000809171028093F1006CCE811175CE009138
:102080007402023008F070CE8091E800877F809360
:10209000E800009371020E94BD08002399F084E0DB
:1020A00080937A0242E061EC81E00E94DC0842E029
:1020B00061EC82E00E94DC0846E261EC83E00E9471
:1020C000DC0852CE8091E30087FDE9CF81E0E8CFC4
:1020D000EF92FF920F931F93CF937C018B010E948D
:1020E0008E08C82F811119C08091E80085FD0DC0B0
:1020F0008091E8008E778093E8000E94620D0E9434
:102100008E08882389F3C82F08C0F70181917F01C9
:102110008093F1000150110939F78C2FCF911F9155
:102120000F91FF90EF900895882341F08095909152
:102130002E03892380932E030C94B90C08958823D1
:1021400039F090912E03892B80932E030C94B90CB7
:1021500008958732D8F58E3108F0FCC08E3009F42E
:102160008FC078F4873009F470C08B3009F456C002
:10217000863009F458C080E695E00E94290580E089
:102180000895863109F4A6C078F48031A1F79091C2
:102190004103892F877F93FF88608093410383FFEA
:1021A0007FC089EE96E063C0893109F47CC08B3131
:1021B00011F790914103892F8D7F91FF8260809369
:1021C000410381FF5AC082E297E051C0883331F168
:1021D00050F4893221F0853311F0873261F680E0C6
:1021E0000E943E0D40C08334D1F320F48A3318F2AC
:1021F0008953F6CF883409F0BECF0E941A0D88E4C7
:1022000097E00E9429052FEF83ED90E32150804055
:102210009040E1F700C000000E94100886EA94E0B8
:102220000E94290520C080914103817F8E7F809389
:10223000410389E395E00E94290589E597E00E9422
:10224000290581E08093400308958091410380FF38
:102250000CC08BE397E00E94290580914103817FA8
:102260008E7F8093410381E008958FE297E00E9482
:102270002905809141038160F4CF84E197E0D0CFBC
:1022800090914103892F8B7F92FF8460809341035B
:1022900082FF03C085E097E0EACF85EF96E0C0CFEC
:1022A0008CED96E0BDCF8DEC96E00E94290588EA82
:1022B00096E00E94290581E696E00E9429058BE3BD
:1022C00096E00E94290586EF95E00E9429058BEC97
:1022D00095E0A6CF8DEB95E00E9429050E94E507C9
:1022E0001F928F9383EA95E09F938F930E94C2057C
:1022F000809112011F928F938CE895E09F938F93AA
:102300000E94C20580913F031F928F9389E795E059
:102310009F938F930E94C2052FB7F89480913B033F
:1023200090913C03A0913D03B0913E032FBFBF931A
:10233000AF939F938F9382E695E09F938F930E9434
:10234000C2058DB79EB742960FB6F8949EBF0FBEDA
:102350008DBF89CF8D5144CFCF93DF93882309F46C
:1023600054C09EE7980F933020F5C2E0D9E382383D
:1023700031F0C4E0D7E4833811F4C1E0D3E50E9422
:10238000E5078C2309F441C08D2F0E9489060E9425
:10239000B90C2FEF41EE54E0215040405040E1F79E
:1023A00000C000008D2F0E947D06DF91CF910C941C
:1023B000B90C9CEF980F913AB0F390E2980F9830D7
:1023C00088F4877021E030E0A90102C0440F551F56
:1023D0008A95E2F7CA01809590912E038923809314
:1023E0002E03E3CF9BE5980F933030F490E080E02C
:1023F000DF91CF910C94DB0B885A873130F490E059
:1024000080E0DF91CF910C94AF0BDF91CF910895D5
:10241000CF93DF93882309F4C2C0C82F8EE78C0FB7
:10242000833030F5C238F1F0C338F9F0C4E0D7E4B6
:102430000E94E5078C2309F0B2C08D2F0E94890607
:102440000E94B90C2FEF81EE94E021508040904023
:10245000E1F700C000008D2F0E947D06DF91CF9133
:102460000C94B90CC2E0D9E3E3CFC1E0D3E5E0CFEF
:102470008CEF8C0F813A08F03FC18091400381308E
:10248000B1F048F0823009F441C0109240038C2F23
:102490000E948906E3CF809136028E3011F087309A
:1024A000B1F78C2F0E94A910811179C0F0CF8091D3
:1024B00036028E30B1F38730A1F3C431C9F048F44D
:1024C000CB3059F0C031C1F087E193E00E9429057B
:1024D00011C0C93269F0C833B9F789E395E00E94A9
:1024E00029058DE193E00E94290581E08170DCCF10
:1024F0001092400380E0FACF0E94070C89E193E03C
:102500000E94290582E080934003EFCFC432D0F4CB
:10251000CE3108F0C0C0CB30E9F048F4C73009F440
:10252000D1C086EC93E0DF91CF910C942905C331A3
:10253000C9F1C431B1F780917F02882349F110922B
:102540007F020AC0CB3409F4BBC0C0F4C93299F38E
:10255000C83339F70E94070C80917F02882309F461
:10256000C8C01F928F9380EC93E09F938F930E943B
:10257000C2050F900F900F900F9011C0C13509F454
:1025800099C0C23509F490C0CE3459F66AE093C0C0
:1025900085ED93E00E94290581E080934003DF915F
:1025A000CF9108958FEA93E00E9429058DE993E089
:1025B0000E942905809118011F928F938AE993E068
:1025C0009F938F930E94C20588E993E00E9429059A
:1025D00086E893E00E942905809117011F928F934E
:1025E00083E893E09F938F930E94C20581E893E074
:1025F0000E94290582E793E00E9429058091160137
:102600001F928F938FE693E09F938F930E94C20552
:102610008DE693E00E9429058CE593E00E94290550
:10262000809115011F928F9389E593E09F938F937B
:102630000E94C20587E593E00E94290582E493E0A9
:102640000E942905809114011F928F938FE393E0DC
:102650009F938F930E94C2058DE393E00E9429050A
:1026600086E293E00E942905809113011F928F93C7
:1026700083E293E09F938F930E94C20581E293E0EF
:102680000E9429058DB79EB748960FB6F8949EBF55
:102690000FBE8DBF61CFCE51EC2FF0E0E75DFE4F56
:1026A000808180937F0258CF61E080917F020E94F9
:1026B0000B0B52CF61E080917F020E948C0A4CCFBD
:1026C0006AE0F3CF8EE18093180182E380931701D3
:1026D0008AE08093160184E18093150188E080935D
:1026E000140188E28093130188EC93E00E9429058D
:1026F00033CF8DEB93E017CF80E28C0F883068F4F6
:10270000C77021E030E001C0220FCA95EAF780913E
:102710002E03822B80932E03A1CE8BE58C0F83306A
:1027200070F481E890E0C53A31F083E890E0C63A71
:1027300011F482E890E0DF91CF910C94DB0B88E5F7
:102740008C0F873108F02BCF82EE90E0C83A09F465
:1027500060C089EE90E0C93A09F45BC08AEE90E06F
:10276000CA3A09F456C085EB90E0CB3A09F451C05F
:1027700086EB90E0CC3A09F44CC083EB90E0CD3A84
:1027800009F447C084EB90E0CE3A09F442C087EBED
:1027900090E0CF3AF1F18CEC90E0C13BD1F18DECBF
:1027A00090E0C03BB1F183E891E0C23B91F18AE84F
:1027B00091E0C33B71F182E991E0C43B51F184E9BE
:1027C00091E0C53B31F181E292E0C63B11F183E239
:1027D00092E0C73BF1F084E292E0C83BD1F085E2A1
:1027E00092E0C93BB1F086E292E0CA3B91F087E209
:1027F00092E0CB3B71F08AE292E0CC3B51F08FE665
:1028000090E0CD3B31F090E080E0CE3B11F480E7EA
:1028100090E0DF91CF910C94AF0BCF92DF92EF92CB
:10282000FF920F931F93CF93DF9300D000D01F929E
:10283000CDB7DEB76C0185E0F601DE01119601909F
:102840000D928A95E1F7F60140815181238134810F
:1028500091E02115310531F05F3F19F491E04F3FD0
:1028600009F090E090FD99C0F6010281F580F294A4
:102870009FE0F92249835A830B83722F3D832C8377
:10288000602F8D810E94A206182FE92FE295EF702C
:10289000EF3008F082C0F0E0E05BFB4E0C946B225E
:1028A0005F145F149D149D1413154515CD14CD149C
:1028B0003716CD140D170D17CD14CD14C917F92FD8
:1028C000FF70FF2E907F19F0F29480EFF822002322
:1028D000C9F0FF2039F080912D03F82AF0922D03E2
:1028E0000E94B90C812F0F900F900F900F900F90B6
:1028F000DF91CF911F910F91FF90EF90DF90CF90DC
:102900000C940812812F0E94AC11FF2009F445C0DD
:10291000F09480912D03F822F0922D030F900F90E8
:102920000F900F900F90DF91CF911F910F91FF901B
:10293000EF90DF90CF900C94B90C892F8F70907F1F
:10294000903211F08295807F112379F0113009F4D3
:1029500049C0002309F455C0FF2059F0F6019581C4
:1029600090FF69C29F70958304C0002321F1F1108C
:102970000FC00F900F900F900F900F90DF91CF919D
:102980001F910F91FF90EF90DF90CF900C949F10CC
:1029900021E0F212EECF80932C030F900F900F9056
:1029A0000F900F90DF91CF911F910F91FF90EF90BB
:1029B000DF90CF900895F11011C010922C030F906A
:1029C0000F900F900F900F90DF91CF911F910F916B
:1029D000FF90EF90DF90CF900C94941091E0F9125B
:1029E000ECCFDBCF002349F0E5E0EF15B0F290919A
:1029F0002E03982309F4BDCFE2CFF4E0FF1568F26F
:102A0000DECFFF20E1F2812F0F900F900F900F90FB
:102A10000F90DF91CF911F910F91FF90EF90DF907A
:102A2000CF900C94AC11892F869586958370C1F058
:102A3000813009F0B2CF812F9370011102C090E074
:102A400080E00F900F900F900F900F90DF91CF913B
:102A50001F910F91FF90EF90DF90CF900C94AF0BF0
:102A6000812F9370011102C090E080E00F900F90D1
:102A70000F900F900F90DF91CF911F910F91FF90CA
:102A8000EF90DF90CF900C94DB0B002309F471C022
:102A9000803FA1F40E9404068195809338030F9033
:102AA0000F900F900F900F90DF91CF911F910F918A
:102AB000FF90EF90DF90CF900C941E0C813F19F4A3
:102AC0000E940406EACF823F31F40E9404068195F9
:102AD00080933703E4CF833F19F40E940406F8CFB4
:102AE000893F29F40E94CB0580933903D8CF8A3FD0
:102AF00021F40E94CB058195F7CF8B3F31F40E94E2
:102B0000CB05819580933A03CACF8C3F19F40E947C
:102B1000CB05F8CF809136038160143FA1F08091FE
:102B200036038260153F79F0809136038460163F4A
:102B300051F0809136038860173F29F0183F31F437
:102B400080913603806180933603A9CF8091300352
:102B500081601D3F59F08091300382601E3F31F04B
:102B60001F3F09F09CCF8091300384608093300335
:102B700096CF803FC1F48091380387FD10923803CF
:102B80008091370381118BCF80913803811187CFDA
:102B900080913903811183CF80913A0381117FCFD6
:102BA000109231037CCF813F29F4809138031816AD
:102BB0002CF3E6CF80913703123F29F487FFE0CF53
:102BC00010923703DDCF133F19F41816CCF3D8CF8A
:102BD000193F39F480913903181694F6109239038D
:102BE000CFCF1A3F29F48091390387FFC9CFF6CFA1
:102BF0001B3F39F480913A0387FFC2CF10923A030A
:102C0000BFCF1C3F29F480913A031816BCF3B8CF0C
:102C1000809136038E7F143FA1F0809136038D7F23
:102C2000153F79F0809136038B7F163F51F08091EC
:102C30003603877F173F29F0183F31F48091360320
:102C40008F7E809336039CCF809130038E7F1D3F13
:102C500059F0809130038D7F1E3F31F01F3F09F006
:102C60008FCF809130038B7F8093300389CF892F62
:102C7000837009F064C0011190CE812F82958695F2
:102C80008770880F880F412F4F70C42ED12CF12CE4
:102C9000E12C082E04C0CC0CDD1CEE1CFF1C0A9499
:102CA000D2F740E050E0BA0114FF11C00FE010E08D
:102CB00020E030E004C0000F111F221F331F8A954F
:102CC000D2F7B901A8014095509560957095009193
:102CD000420310914303209144033091450396959C
:102CE000969593709230E9F028F5913089F04C294F
:102CF0005D296E297F29402351236223732340934A
:102D0000420350934303609344037093450345CEBD
:102D1000C02AD12AE22AF32A4C295D296E297F296B
:102D2000EECF4C295D296E297F2940275127622744
:102D30007327E5CF4023512362237323EDCF86957C
:102D4000002311F0892F8170882309F426CE812F6A
:102D5000829586958770880F880F412F4F70C42EFB
:102D6000D12CF12CE12C082E04C0CC0CDD1CEE1C67
:102D7000FF1C0A94D2F740E050E0BA0114FF11C0E2
:102D80000FE010E020E030E004C0000F111F221F10
:102D9000331F8A95D2F7B901A801409550956095E7
:102DA00070950091B8021091B9022091BA02309149
:102DB000BB029695969593709230E9F028F5913084
:102DC00089F04C295D296E297F29402351236223F4
:102DD00073234093B8025093B9026093BA02709380
:102DE000BB02DBCD0C291D292E293F29402B512B5D
:102DF000622B732BEECF4C295D296E297F2940274A
:102E0000512762277327E5CF402351236223732381
:102E10004C295D296E297F29DCCF803F09F44EC003
:102E2000D0F480E4810F803270F1002309F4ACC04B
:102E3000FF2009F4A6C0812F0E940812193309F05F
:102E400099C0FFEF21EE84E0F15020408040E1F78F
:102E500000C00000A2CD823F09F470C008F45BC03E
:102E6000833F19F7002309F47CC0292F2F7181E0DB
:102E700090E0A0E0B0E004C0880F991FAA1FBB1F1C
:102E80002A95D2F73AC0E12FE071FE2E892F8F717B
:102E9000002351F00E946F07812F8295807FF110EF
:102EA00068CD812F8F7065CD0E944B07812F829551
:102EB000807FF11084CD812F8F7081CD002331F17F
:102EC000F4E0FF1508F469CD292F2F7181E090E01F
:102ED000A0E0B0E004C0880F991FAA1FBB1F2A956D
:102EE000D2F74091B8025091B9026091BA02709144
:102EF000BB0284279527A627B7278093B802909313
:102F0000B902A093BA02B093BB0247CD25E02F15BA
:102F100008F443CDD9CF892F8F71002399F00F90FA
:102F20000F900F900F900F90DF91CF911F910F9105
:102F3000FF90EF90DF90CF900C946F07892F8F71E7
:102F4000002369F30F900F900F900F900F90DF9177
:102F5000CF911F910F91FF90EF90DF90CF900C9445
:102F60004B071092B8021092B9021092BA02109256
:102F7000BB0213CD133509F464CF173409F00DCD1E
:102F800060CF892F8F71CBCFF1103DCD892F8F71FD
:102F9000D9CF811102CD002309F4FFCC0E941A0D74
:102FA0008FEF90E7E2E081509040E040E1F700C011
:102FB00000000E9410080F931F93CF93DF9380911E
:102FC0008502807FB9F480918202882399F08091F4
:102FD000B702109186026091800270918102C091C7
:102FE0008302D091840221E06F3F09F020E006E0E7
:102FF000181305C0DF91CF911F910F91089531E013
:10300000209721F0322F7F3F09F030E090E030FD33
:1030100033C0089FF001099FF00D1124DF01A9576B
:10302000BD4F11963C911197371326C03C91361332
:1030300023C012963C91129731111EC013964D91E8
:103040005C914C1B5D0B483C5105B0F480918502AE
:103050008F70806180938502E457FD4F80818F706F
:103060008061808380E892E00E940D14DF91CF910F
:103070001F910F910C948F0701968770B9CF9F9283
:10308000AF92BF92CF92DF92EF92FF920F931F9376
:10309000CF93DF93CDB7DEB761970FB6F894DEBF5D
:1030A0000FBECDBF8C0185E0F801DE011D960190B9
:1030B0000D928A95E1F7F80140815181F280C38039
:1030C000D48090918002609181022091830230919E
:1030D000840281E02115310531F06F3F19F481E060
:1030E0009F3F09F080E0F82FF1709F2E80FD49C1CD
:1030F00080E8A82E82E0B82EE0908202F601E21B62
:10310000F30BEE2009F400C180918502782F707FC7
:10311000E83CF10508F0BAC0711181C0EF2C6513CD
:1031200022C0941320C0F1101EC08F708061809364
:103130008502C5010E940D1480918502F8018583E6
:103140008E2D61960FB6F894DEBF0FBECDBFDF9116
:10315000CF911F910F91FF90EF90DF90CF90BF9094
:10316000AF909F90089581E0C114D10431F05F3F8A
:1031700019F481E04F3F09F080E080FD24C081E038
:103180008F25F82FF170BF2E80FF3FC08091B702CE
:103190002091860236E0821318C07C2DD98AC88A15
:1031A0006F2D89890E94A206292F22952F70223027
:1031B00000F1243028F59F7001F1F8019581907F8E
:1031C000E1F4E92CBDCF80E0DCCF90E0389FF00146
:1031D000399FF00D1124E957FD4F6181561306C048
:1031E0006081461303C062816F110FC00196877022
:1031F000D2CF9F7011F0882321F3805E883008F3CE
:10320000C8010E940D149B2CDCCFFF2009F498CF3D
:1032100080918502816080938502E12C91CF6513B6
:1032200006C0941304C0F801FF2009F488C04D873C
:103230005E87FF867C2DD98AC88A6F2D89890E9476
:103240009907882309F4ABC0FF2009F4A8C0809136
:103250008502803270F0209180023091810238879F
:103260002F831986DB86CA868C87CE0107960E943B
:103270000D1486E0F801A0E8B2E001900D928A9565
:10328000E1F70E94DB17EE24E3945ACF71110AC0D4
:1032900080E892E00E940D1486E0F50111928A9573
:1032A000E9F7BBCF65130FC094130DC0F1100BC02D
:1032B000F8018583C8010E940D1486E0F501119282
:1032C0008A95E9F73DCF4D875E87FF867C2DD98AA9
:1032D000C88A6F2D89890E949907882309F45FC0E5
:1032E000FF2009F45CC080918502803210F22091A9
:1032F0008002309181023A8329831B82DD82CC8255
:103300008E83CE010196B3CFE83CF105B0F6EF2CE9
:10331000FF2009F444C065131FC094131DC08091A1
:10332000850280FD10C0982F907F69F0F801858399
:10333000903F31F0982F907F905F8F70892B85831D
:10334000C8010E940D1486E0F801A0E8B2E00190E7
:103350000D928A95E1F7F4CE4D875E87FF867C2D2E
:10336000D98AC88A6F2D89890E949907811181CFD6
:1033700080918502816080938502C8010E940D14AE
:10338000DFCEFF2061F04D875E87FF867C2DD98AD6
:10339000C88A6F2D89890E94990781116ACFC80157
:1033A0000E940D1470CF1F93CF93DF93CDB7DEB77C
:1033B00067970FB6F894DEBF0FBECDBF4B8B5C8B0B
:1033C0006D8B7E8B8F8B1A8A198A85E0FE0173962E
:1033D000DE011D9601900D928A95E1F786E0FE01CF
:1033E0003D96DE01179601900D928A95E1F7CE0188
:1033F00007960E943F18811137C086E0FE0137967C
:10340000DE01119601900D928A95E1F79F818885E2
:103410002A853B85232B39F08F3F19F481E09F3FAC
:1034200019F080E001C081E080FD1EC0209186027D
:1034300030E0C9010196877099274091B70248177B
:10344000190659F196E0929FD001939FB00D112477
:10345000A957BD4FFE01319601900D929A95E1F763
:10346000809386020E948F0716E08091B7029091A8
:1034700086028917F9F0819FC001112489579D4F59
:103480000E943F188823B1F08091B70290E0019626
:10349000877099278093B702E8CF0E941A0D109287
:1034A00086021092B70286E0E0E8F2E0DF011D92AA
:1034B0008A95E9F767960FB6F894DEBF0FBECDBFC9
:1034C000DF91CF911F910895CF93DF9300D01F928A
:1034D000CDB7DEB720917A02243021F523E029838D
:1034E0009B838A8382E08093E9008FEF9091E800CC
:1034F000815095FD06C095ED9A95F1F70000811178
:10350000F5CF8091E80085FF0DC050E040E063E01A
:1035100070E0CE0101960E9468108091E8008E77DD
:103520008093E8000F900F900F90DF91CF91089556
:10353000CF93DF9300D01F92CDB7DEB720917A02F0
:10354000243061F519821A821B8222E02983813896
:10355000910520F0805891099B838A8382E08093B3
:10356000E9008FEF9091E800815095FD06C095ED40
:103570009A95F1F700008111F5CF8091E80085FF61
:103580000DC050E040E063E070E0CE0101960E9483
:1035900068108091E8008E778093E8000F900F907C
:1035A0000F90DF91CF91089520917A02243049F550
:1035B00022E02093E9002FEF3091E800215035FD03
:1035C00006C035ED3A95F1F700002111F5CF2091B5
:1035D000E80025FF16C02091110150E040E063E0B3
:1035E00070E0222339F021E02093F10050E040E028
:1035F00065E070E00E9468108091E8008E7780930B
:10360000E8000895CF93DF9320917A02243011F5DA
:1036100021E02093E90021E8215021F03091E800D9
:1036200035FF1BC02091E80025FF14C0EC0150E0DD
:1036300040E068E070E00E9468108091E8008E77BA
:103640008093E80088E0FE01A7E6B2E001900D92C9
:103650008A95E1F7DF91CF910895EFE3F1E031979B
:10366000F1F700C00000D8CF5198599A85E08A95AB
:10367000F1F7000089B1869581700895CF93DF93AB
:10368000EC010E94341B882311F0209721F4CE0115
:10369000DF91CF91089585E08A95F1F70000219799
:1036A000F0CF0F931F93CF93DF9310924102CAEF95
:1036B000D0E088EE93E00E943E1B892B21F42197F5
:1036C000C1F781E00AC0D8E0C0E0CC0F88EC90E000
:1036D0000E943E1B892BB9F582E08093410287ED61
:1036E00091E00E942905809141021F928F9382ED03
:1036F00091E09F938F930E94C20580ED91E00E941C
:1037000029059FEF29E688E1915020408040E1F7AC
:1037100000C000000E947D0A0E94770A0F900F905F
:103720000F900F90CFEF23C025E02A95F1F700000E
:10373000015011090E94341B811108C001151105A7
:1037400099F783E0CACF08EC10E0F4CF012BC9F35E
:103750005098589A85E08A95F1F700004899C16021
:10376000D15009F0B2CF0E947D0A0E94770A8C2FB7
:10377000DF91CF911F910F910895EF92FF920F93D8
:103780001F93CF93DF93E82E109241020E947D0A8F
:103790000E947A0ACAEFD0E088EE93E00E943E1BB6
:1037A000892B21F42197C1F781E00BC008E010E0DC
:1037B00080E8F82E8AEF90E00E943E1B892B41F5AD
:1037C00083E0809341028FEB91E00E942905809174
:1037D00041021F928F938AEB91E09F938F930E94F7
:1037E000C20588EB91E00E9429059FEF29E688E158
:1037F000915020408040E1F700C000000E947D0A07
:103800000E94770A0F900F900F900F9080E02AC0CF
:103810008E2D8F2161F00E94770AC8ECD0E00E94C3
:10382000341B81110DC0209729F484E0CACF0E9477
:103830007A0AF3CF25E02A95F1F700002197EFCF20
:10384000CD2B99F3F6940150110909F0B3CF8FE80D
:1038500091E00197F1F700C000000E947D0A0E94EC
:10386000770A81E0DF91CF911F910F91FF90EF9048
:103870000895CF9384E10E94BD1B0E94511BC82F65
:103880008B37C1F08091410380FF0CC01F92CF9312
:103890008AEE91E09F938F930E94C2050F900F9044
:1038A0000F900F908091410380FF04C088EE91E05B
:1038B0000E9429058C2FCF9108951F93CF93DF93FA
:1038C000809100018F3FD1F486E10E94BD1B0E94D0
:1038D000511B809300018F3F29F480E0DF91CF914D
:1038E0001F9108951F928F938BEA91E09F938F937E
:1038F0000E94C2050F900F900F900F90C091400250
:10390000CC2351F010924002CB3739F3CF3F09F06E
:103910008BC0C0930001E1CFC0913F02CC2319F0CE
:1039200010923F02F1CFC0913E02CC23E1F0109201
:103930003E028C2F8F77813721F1893779F50E94EC
:10394000391CC82F8F778D3019F088F4853099F4A1
:103950008C2F0E94800AC7FF0EC0C82FC0648066EB
:1039600080934002D1CF0E94391CC82FE2CF813111
:1039700079F38B3169F38C2F0E94800AC82FC064C1
:10398000C3CF0E94391C982F9F77913729F0993720
:1039900051F00E94800A30C080933E028C2F0E941A
:1039A000800AC82FB1CF0E94391CD82F8F778D3055
:1039B00019F0D0F48530E1F4C7FF21C08C2F0E94AC
:1039C000800AC82F87E991E0D7FF2BC08CE991E0EE
:1039D0000E942905C0933F028D2F0E94800A982FD4
:1039E000906690934002CACF813131F38B3121F33D
:1039F0008D2F0E94800A806480934002CFCF8D2F4C
:103A00000E94800A182FC82FC0668DE891E0D7FF6A
:103A100008C082E991E00E942905C0934002C12FAD
:103A2000AECF0E94290570CF2091510230915202F1
:103A3000EC2FE695E695E6954C2F477081E090E0F7
:103A400001C0880F4A95EAF7C7FF22C0EF70E20F66
:103A5000F32FF11D8095908189238083809141030C
:103A600080FF14C089EA91E00E9429051F92CF933C
:103A700084EA91E09F938F930E94C20581EA91E0CE
:103A80000E9429050F900F900F900F9081E026CF94
:103A9000E20FF32FF11D9081892BDFCF78941F92D5
:103AA0000F920FB60F9211248F939F93AF93BF93F2
:103AB00080913B0390913C03A0913D03B0913E0364
:103AC0000196A11DB11D80933B0390933C03A093ED
:103AD0003D03B0933E03BF91AF919F918F910F90A3
:103AE0000FBE0F901F9018951F920F920FB60F9256
:103AF00011248F939F93AF93BF9380912F038111D4
:103B000013C080913B0390913C03A0913D03B09181
:103B10003E034196A11DB11D80933B0390933C034E
:103B2000A0933D03B0933E03BF91AF919F918F91BE
:103B30000F900FBE0F901F9018951F920F920FB607
:103B40000F9211242F933F934F935F936F937F9323
:103B50008F939F93AF93BF93EF93FF938091E10077
:103B600082FF09C08091E20082FF05C08091E100E0
:103B70008B7F8093E1008091DA0080FF1FC08091ED
:103B8000D80080FF1BC08091DA008E7F8093DA001E
:103B90008091D90080FF9DC080E189BD82E189BD0F
:103BA00009B400FEFDCF81E080937A028091640227
:103BB000811104C00E94F1070E940E098091E1006A
:103BC00080FF1FC08091E20080FF1BC08091E20057
:103BD0008E7F8093E2008091E20080618093E2001A
:103BE0008091D80080628093D80019BC85E08093D2
:103BF0007A028091660280936502109266020E94AA
:103C00001A0D8091E10084FF2DC08091E20084FFB5
:103C100029C080E189BD82E189BD09B400FEFDCFE4
:103C20008091D8008F7D8093D8008091E1008F7EB5
:103C30008093E1008091E2008F7E8093E20080918A
:103C4000E20081608093E20080917102882309F490
:103C500046C084E080937A020E941A0D809165022A
:103C6000809366028091E10083FF22C08091E20090
:103C700083FF1EC08091E100877F8093E10082E096
:103C800080937A02109271028091E1008E7F80937E
:103C9000E1008091E2008E7F8093E2008091E2005B
:103CA00080618093E20042E060E080E00E94DC08F6
:103CB000FF91EF91BF91AF919F918F917F916F9104
:103CC0005F914F913F912F910F900FBE0F901F90DA
:103CD000189519BC10927A02109264026FCF8091ED
:103CE000E30087FD02C081E0B5CF83E0B3CFCF937F
:103CF000DF93CDB7DEB72B970FB6F894DEBF0FBEBC
:103D0000CDBF84B7877F84BF0FB6F894A895809104
:103D10006000886180936000109260000FBE80E8B0
:103D200090E00FB6F89480936100909361000FBE0D
:103D30008AE899E0909335018093340187E091E01F
:103D4000909333038093320382E392E00E9429052B
:103D50000E94F1070E940E09789482E084BD93E0EE
:103D600095BD9AEF97BD80936E008091410381606D
:103D7000809341030E947D0A0E94770A2FEF83ED12
:103D800090E3215080409040E1F700C00000E3E460
:103D9000F2E081E592E011928E179F07E1F783E44C
:103DA00092E09093520280935102569A5E9AEFEFFE
:103DB000F9E628E1E150F0402040E1F700C00000C2
:103DC000569A5E9880917A02843009F036C10E943A
:103DD0007209882309F431C180E292E00E9429052A
:103DE00082E192E00E942905F9E14F2EF1E05F2E79
:103DF000AFEE6A2EA1E07A2EB7E0AB2EB2E0BB2E7A
:103E000018E1812E912C80917A02853009F418C135
:103E10000E945D1CE4E5CE2EE2E0DE2EF12CE12CCA
:103E2000EB86E0915102F0915202EE0DFF1D3080C1
:103E3000F6012080231409F45FC08091410381FFC3
:103E400038C08AEF91E00E94290510E000E0E0917F
:103E50005102F0915202E00FF11F2081229530E0D3
:103E6000C901880F991F880F991F8C7C359527955C
:103E7000359527952373822B90E05F924F929C019A
:103E8000220F331F2A7A959587958575822B1F926D
:103E90008F931F930F937F926F920E94C2050F5FC3
:103EA0001F4F0FB6F894DEBF0FBECDBF0E30110509
:103EB00071F600E011E02324822D8123C9F00E83E6
:103EC0009B859F8391E0812F832109F490E098875F
:103ED0000E9471068160782F9A8789874E815F8161
:103EE00068858A850E94D319F601808181278083A5
:103EF0000F5F110F083001F7FFEFEF1AFF0A2FEFE6
:103F0000C21AD20A8EE0E816F10409F089CF9FEFB9
:103F100099839A831B820E9471068160782F9D830A
:103F20008C8349815A816B818D810E94D3192091A4
:103F30003403309135034FB7F89480913B0390914F
:103F40003C03A0913D03B0913E034FBFAC01421B27
:103F5000530B809131032091170130E0811106C08D
:103F600020911801EAE02E9F900111244217530777
:103F700080F090913703F09038031091390300914D
:103F80003A03911197C0F1105DC111115BC101118C
:103F900059C10E94E507909153028917C9F00E9408
:103FA000E50780935302909141039570953051F449
:103FB0001F928F93BF92AF920E94C2050F900F90F5
:103FC0000F900F9080915302569A81FFE1C05E9A44
:103FD0002091E4003091E5008091620290916302AB
:103FE0002817390739F18091E4009091E50090930A
:103FF0006302809362020E9472098823D9F0809143
:104000007A028430B9F48091E9008F709091EC00CD
:1040100090FFC0C090E8892B93E09093E9009091C5
:10402000EB0090FF04C09091EE0097FDD1C08F701F
:104030008093E9000E94620DE6CE0E94620DC2CE1E
:1040400080917A02843011F110922F0380E40FB630
:10405000F894A895809260000FBE8093600083B7AB
:10406000817F846083BF83B7816083BF78948895A4
:1040700083B78E7F83BF0FB6F894A89580916000B8
:10408000886180936000109260000FBE8091700282
:10409000882309F4B8CE0E945D1CE0915102F09192
:1040A0005202CF010E9621912111B6C08E179F07A3
:1040B000D1F7A9CE8F3F19F08F5F80933103191686
:1040C00024F40E940406809337038091370387FF0E
:1040D00005C00E9404068195809337031F1424F4C1
:1040E0000E940406809338038091380387FF05C03F
:1040F0000E940406819580933803609137036623FC
:1041000031F1F0903803FF2011F1062E000C770BEF
:10411000880B990B0E945E2123E333E343E35FE3C3
:104120000E94C2210E942621609337036F2DFF0C4D
:10413000770B880B990B0E945E2123E333E343E363
:104140005FE30E94C2210E9426216093380311166A
:1041500024F40E94CB05809339038091390387FFB3
:1041600005C00E94CB05819580933903101624F475
:104170000E94CB0580933A0380913A0387FF05C0E4
:104180000E94CB05819580933A030E941E0C01CFBB
:104190005E981ECF90E03FCFE0910201F0910301C5
:1041A000E90FF11D20819F5F3091060193239093C9
:1041B00005012093F1009091E80095FD09C09091D0
:1041C000E80090FF05C09091E8009E779093E8008A
:1041D0009091050120910401291721F02091E80018
:1041E00025FDDACF2091F3009091F200322F292F94
:1041F000232B09F41CCF9091E80090FF18CF9091E9
:10420000E80095FD06C09091E8009E779093E80045
:104210000ECF1092F100F3CF80E189BD82E189BD1C
:1042200009B400FEFDCF8091D8008F7D8093D80027
:104230008091E00082608093E0008091E00081FD49
:10424000FCCFE1CD8F3F09F037CF48CF0E942D2121
:104250006894B1110C94BC2108950E94A12188F0AA
:104260009F5798F0B92F9927B751B0F0E1F0660F3A
:10427000771F881F991F1AF0BA95C9F714C0B1307B
:1042800091F00E94BB21B1E008950C94BB21672FEF
:10429000782F8827B85F39F0B93FCCF386957795AA
:1042A0006795B395D9F73EF4909580957095619593
:1042B0007F4F8F4F9F4F0895E89409C097FB3EF4BE
:1042C00090958095709561957F4F8F4F9F4F992363
:1042D000A9F0F92F96E9BB279395F69587957795E1
:1042E0006795B795F111F8CFFAF4BB0F11F460FFA1
:1042F0001BC06F5F7F4F8F4F9F4F16C0882311F0F9
:1043000096E911C0772321F09EE8872F762F05C00C
:10431000662371F096E8862F70E060E02AF09A95A7
:10432000660F771F881FDAF7880F9695879597F99C
:10433000089557FD9058440F551F59F05F3F71F095
:104340004795880F97FB991F61F09F3F79F08795FC
:104350000895121613061406551FF2CF4695F1DF85
:1043600008C0161617061806991FF1CF8695710515
:10437000610508940895E894BB2766277727CB0149
:1043800097F908950E94D5210C9446220E94382264
:1043900038F00E943F2220F0952311F00C942F2238
:1043A0000C94352211240C94BC210E94992170F3A5
:1043B000959FC1F3950F50E0551F629FF001729FCA
:1043C000BB27F00DB11D639FAA27F00DB11DAA1FD9
:1043D000649F6627B00DA11D661F829F2227B00D26
:1043E000A11D621F739FB00DA11D621F839FA00DB1
:1043F000611D221F749F3327A00D611D231F849F01
:10440000600D211D822F762F6A2F11249F57504057
:104410009AF0F1F088234AF0EE0FFF1FBB1F661FD2
:10442000771F881F91505040A9F79E3F510580F09B
:104430000C942F220C94BC215F3FE4F3983ED4F3FC
:10444000869577956795B795F795E7959F5FC1F73F
:10445000FE2B880F911D9695879597F9089597F9EA
:104460009F6780E870E060E008959FEF80EC08951A
:1044700000240A9416161706180609060895002443
:104480000A9412161306140605060895092E0394BD
:10449000000C11F4882352F0BB0F40F4BF2B11F431
:1044A00060FF04C06F5F7F4F8F4F9F4F089597FB52
:1044B000072E16F4009407D077FD09D00E947122D0
:1044C00007FC05D03EF4909581959F4F0895709517
:1044D00061957F4F0895EE0FFF1F0590F491E02D39
:1044E0000994AA1BBB1B51E107C0AA1FBB1FA6173B
:1044F000B70710F0A61BB70B881F991F5A95A9F78D
:0E45000080959095BC01CD010895F894FFCFF1
:10450E00FF0536010000FF6F09021BD41A981A64CA
:10451E001A01012808140A321E00407F224D01CED6
:10452E0000AC005D0276028F02010203040506074D
:04453E000809000068
:106800000000000000000000040005000600070072
:10681000080009000A000B000C000D000E000F001C
:1068200010001100120013001400150016001700CC
:10683000180019001A001B001C001D001E001F007C
:10684000200021002200230024002500260027002C
:10685000280000002A002B002C002D002E002F0005
:10686000300031A1320033003400350036003700EB
:106870003800E00000000000000000000000000000
:106880000000000000000000000000000000000008
:1068900000000000000000000000000000004F00A9
:1068A000500051005200530067005400550056003C
:1068B000580059005A005B005C005D005E005F00FC
:1068C0006000610062006300640000005700000087
:1068D00000000000000000000000000000000000B8
:1068E00000000000000000000000000000000000A8
:1068F0000000E100E200E300000000000000F1A160
:106900000100010001000100EA4401000100E2442D
:106910000100010001000100460001004A004B0097
:10692000010001004700480001000100E9440100A6
:106930000100010001000100010001003A003B00DC
:106940003C003D003E003F0040004100420043004B
:10695000010000004C00010001004400450052000D
:1069600049000100010050004F0029004D004E0079
:1069700051000100010001000100010001000100BF
:1069800001000100010001000100010001000100FF
:1069900001000100010001000100010001004D00A3
:1069A0004A004E004B0001000100010001000100FF
:1069B00001000100010001000100010001000100CF
:1069C00001000100010001000100010001000100BF
:1069D00001000100010001000100010001000100AF
:1069E000010001000100010001000100010001009F
:1069F000010001000100010001000100010001008F
:00000001FF
